:030000000219FDE5
:03000B000200AA46
:03002B000201557A
:03005B000202E9B5
:030073000202D6B0
:1000800002030406080C10182030406080040608A3
:100090000C10182030406080A0C00003070F1F0D17
:1000A0000D04050D050305030302C2AFC0D0C0E077
:1000B000206214E5256009E473E525F4F58AD2622F
:1000C000D0E0D0D0D2AF3285268AC262E526F46075
:1000D0003130682720720CE57BF45290D0E0D0D00C
:1000E000D2AF32E57BF45290206F1020650DE57B96
:1000F000F4D33333335290E57B4290D0E0D0D0D26A
:10010000AF32758A00C28DD26201FB01B930680737
:10011000206504D295D29201B9306807206504D2D7
:1001200094D29101B9306807206504D293D290012E
:10013000B9306807206504D295D29201B9306807BA
:10014000206504D294D29101B9306807206504D2A9
:1001500093D29001B9C2AFC2AD53E6EFC0D0C0E0B8
:10016000D2D3D2AFC2CEE52A6007207449152A2126
:10017000B67800790020742EE580307E01F430E7F7
:100180000278FF53DACF207E0343DA20307E034328
:10019000DA10C2D8C271E580307E01F430E702790E
:1001A000FFC3E89970CB306103752A18207403757A
:1001B0002A18885CD27020740DE52B6004152B2161
:1001C000C643DA01C2D82070024135A85C20610222
:1001D000C2702074367982B70431C3E894F04003CA
:1001E00074F0F8E8C4540F28F87984B70302410B7F
:1001F000C313C3138721200802C313200A06C3C8F0
:1002000098F8410B28F8500374FFF88822E52D5424
:10021000066022206B1FE536C333C333F8E564C3A1
:1002200013C313F9C3952240028922E82522F5223F
:1002300050037522FF7882B60459852224A824C36E
:10024000E52495614002A861C3E895634002A86374
:100250008825E56670024186C3E8AA669A5003E8DD
:10026000FAE4F9EAC333FBE568F45B29400D25673E
:10027000F8E56760021567400B41860AC3E5679A97
:100280005002056778FF8826C26FC3E52694F840C0
:1002900002D26F20CF0AD0E0D0D043E610D2AD32E8
:1002A000C2CF053A7801E52A6005307402152AC3E9
:1002B000E55C94014005755F0041CC75600075698F
:1002C00000E55F2401F55F5003755FFFD0E0D0D0FB
:1002D00043E610D2AD32C2AF53E67F7592FA759302
:1002E000FFC260759104D2AF32C2AF53E6EFC2AD28
:1002F000C0D0C0E0C0F0D2D3D2AFA8FBA9FCC2D816
:10030000307102615053DACF207E0343DA10307E21
:100310000343DA20D271E580307E01F420E70261E8
:100320002788278928A17D53DACF207E0343DA204E
:10033000307E0343DA10C2D8C271307402A16978EA
:1003400000E580307E01F430E702A169885CA151AC
:1003500053DACF207E0343DA20307E0343DA10C223
:1003600071206102812953DACF207E0343DA1030F5
:100370007E0343DA20C2D8D27188578958C3E895E2
:1003800055F8E99556F97B007E087A00C3E8948C0D
:10039000E994005005755B00811B882178A2E6A8CE
:1003A000216055C3E894C8E994005008E4D2E4FB06
:1003B0007A0A61F6C3E89468E994015008E4D2E34C
:1003C000FB7A0F61F6C3E894D0E994025008E4D2B6
:1003D000E2FB7A1E61F6C3E894A0E994055008E4B4
:1003E000D2E1FB7A3C61F6C3E89498E9940850089E
:1003F000E4D2E0FB7A787E00C3E89559FCE9955A8F
:10040000FD30E70AECF42401FCEDF43400FD755BEB
:1004100000C3EC9AED9E5003755B018859895A859B
:1004200057558558567802A151C3E89527F8E995A4
:1004300028F9307C02A135307B02A135307A02A147
:100440002E207502814CE9FDE8FC816BE9C313F9AC
:10045000E813F8307902A12EE9C313F9E813F83054
:100460007802A12EE9C313FDE813FC20612CC3EC34
:0E047000941CED940240028182ED701EC3ECDC
:10047E0094C850180529E52970021529C3E5299459
:10048E000A5002A169755C00D270A169E52960026B
:10049E0015297888E6F97400207F087896B903024A
:1004AE00789EE624FAFEE43400FFC3EC9EFCED9F3A
:1004BE00FD9208B90310A2085007207609D2768162
:1004CE00D4307602C276A2085016B9030DECF4248D
:1004DE0001FCEDF43400FD0204EE78007900A13544
:1004EE00B90315EC33FCED33FDC3EC940AFCED942B
:1004FE0000FD50047C007D00C3EC94FFED940040A1
:10050E000678FF7900A135EC8572F0A4C5F0A2F74C
:10051E0033F87900400302055178FF790002055146
:10052E00E9C313F9E813F8307C0EE9600278FFC3D3
:10053E00E81338F8E43400F9C3E894FFE994004076
:10054E000278FF885CD270206102A169741FF45595
:10055E002F4BF52FC274EB7002D274752A183074BB
:10056E0003752A0A306102A17D20740353DAFE203E
:10057E007403752B06D0F0D0E0D0D0D2AD43E61088
:10058E003279010205AD79030205AD790A0205AD96
:10059E00791E0205AD79640205AD79C80205AD7804
:1005AE0017E4D5E0FDD8FAD9F6227A147B78020545
:1005BE00D47A107B8C0205D47A0D7BB40205D47AE2
:1005CE000B7BC80205D4E573D5E001227902E4C2A3
:1005DE0091D5E0FDD294D291D5E0FDC291D5E0FD4A
:1005EE00C294D291D5E0FDE920E004D295D29230AA
:1005FE00E004D293D290E573D5E0FDE920E002C28B
:10060E009230E002C2907496D5E0FDD9C1EAF8D5D9
:10061E00E0FDD8FBDBB0C29122C37C007D0075F0FB
:10062E000005F0EA33FAEB33FB50F6EB13FBEA135B
:10063E00FAC3E9FFE8FEE89AF8E99BF95004EFF9EE
:10064E00EEF8B3EC33FCED33FDD5F0DFEDF9ECF85D
:10065E0022E889F08A20D2D4F8A9F07B0030F70B7B
:10066E007BFFF42401F8E9F43400F9E88520F0A4C6
:10067E00ADF0F8E98520F0A4AFF0FEED2EF9740090
:10068E003FFA7C04C3EA13FAE913F9E813F8DCF431
:10069E008BF030F70AE8F42401F8E9F43400F9E8B5
:1006AE0089F0C2D4F8A9F0227882B60403020711A9
:1006BE00C3E55C940140030206DB852224E4F54485
:1006CE00F545F546F547F548C26E0207117882E604
:1006DE00FCD26EE522F523783879C7AA40AB41C328
:1006EE00EB13FBEA13FAEC146013C3EB13FBEA13E0
:1006FE00FAEC14146007C3EB13FBEA13FAD1278844
:10070E0044894522C3E5449523F8E5459400F95004
:10071E000CC3E89480E994FF4016020742C3E894A4
:10072E007FE994005003020742787F790002074266
:10073E00788079FF8849894A22E5492546F8E54AB5
:10074E003547F9854A20E4300701F43548FA30E799
:10075E0009C3EA94F04015020780C3EA940F5003D0
:10076E0002078078FF79FF7A0F0207807800790000
:10077E007AF0C3E5249561500AC374019524500B99
:10078E0002079EE54A20E70E02079EE54A30E7067D
:10079E00884689478A482278A5E6FAC3E54933F8A0
:1007AE00E54A33F9D15FE930E70BC3E89480E99469
:1007BE00FF4013E1D8C3E8947FE994005002E1D8DA
:1007CE00787F7900E1D8788079FFE820E715C3E5D6
:1007DE002398F84009C3E8940140030207FF78010B
:1007EE000207FFE8F424012523F840030207FF78EF
:1007FE00FF884B2278A6E6FAA847A94812065FE9B9
:10080E0030E70CC3E89401E994FF4016020834C3A4
:10081E00E894FFE99400500302083478FF7900024F
:10082E000834780179FFE920E715C3E54B98F840C5
:10083E0009C3E89401400302085B780102085BE8F3
:10084E00F42401254BF8400302085B78FF8824222C
:10085E0078FF20692879A1E76023E541601F74FFC6
:0F086E008541F0848539F0306A0375F005A4F8F0
:10087D00C5F0600278FFC3E895645002A8648863F0
:10088D0022C3E5409440E5419401E5635003140112
:10089D009F046002F563220208A72275E890227872
:1008AD0083E6FF30EDF9A8BDA9BE0570C3E57094D0
:1008BD00084052757000E9FA79A0E76044EA7007C4
:1008CD00E571601B0208E0C3E895716010E5715099
:1008DD0006600C140208EC0460F90208ECE571F5F1
:1008ED0071C39472401B7561C0C39404401375614C
:1008FD0080C39404400B756140C39404400375613B
:10090D000075BB0E22E5612410500274FFF561796C
:10091D0082B704022139C3A861E524985002A824A6
:10092D00C3E895634002A86388258826E570B4075F
:10093D000375BB1022743279A787F0A4C5F0A2F716
:10094D0033F8C3E895614002A86188228824882580
:10095D0088268864227540007541F022C2AF75C8A3
:10096D0020A8CCA9CDAA3A30CF010A75C824D2AFA0
:10097D00AB3BAC3C883B893CC3E89BF8E99C2069C8
:10098D0008F9306602417821D2AD3D8A3DF9EA9DE4
:10099D00FA600478FF79FFAE3EAF3F8B3E8C3FA8E7
:1009AD003BA93CC3E89EF8E99FF9C3E54113FBE57C
:1009BD004013FAE82AF540E93BF54150067540FF32
:1009CD007541FF411FAA40AB41AC40AD417E047F54
:1009DD0002C3EB9404400D1E1FC3EB940840052089
:1009ED006A021E1FC3ED13FDEC13FCDEF7C3EA9C78
:1009FD00FAEB9DFBEF6009C3E913F9E813F8DFF794
:100A0D00EA28FAEB39FB8A408B4150067BFF8B407D
:100A1D008B41C3EB94025002D2663069047F0341CF
:100A2D004A7892E6FFC3E537948240110FC3E5374C
:100A3D0094A040010FC3EF940640027F057E02E5AE
:100A4D0041C4540FF9E541C454F0F8E540C4540FC6
:100A5D0028F8C3E89EFAE99400FB4009C3EA940222
:100A6D00EB940050047A02E4FB41C4AA40AB41EB85
:100A7D00C4FEEAC4540F4EFCC3EA9CFAEB9400FB8F
:100A8D00C3E813C313F8EA28FAEB3400FB8A408B52
:100A9D0041C3EB94024002C2667802EBC4FE7B00B8
:100AAD00EAC4540F4EFAC3EA98FA4005C3940250B3
:100ABD00027A027892E6FF30600241C48551928538
:100ACD005293D26043E680C3E49AF8E49BF9306612
:100ADD00026150E8FAE9FBD3E913FDE813FC8851F4
:100AED008952C3EF94036038EF20E00DE82CF8E94C
:100AFD003DF9ECFAEDFB020B19E828F8E939F9C3D9
:100B0D00E82402F8E93400F97AFE7BFFC3EF940381
:100B1D00400E8A538B54884D894E8C4F8D50618475
:100B2D00885389548A4D8B4E8C4F8D503069127578
:100B3D0053F07554FF754FF07550FF7551F07552A8
:100B4D00FF6184E8FAD3E813FC8851C3EF94036086
:100B5D0020EF20E007E82CF8ECFA6170E828240279
:100B6D00F87AFEC3EF940340088A53884D8C4F6189
:100B7D008488538A4D8C4FE568C3335002646BF5FE
:100B8D0068306002618E753402D26043E680E52DD7
:100B9D0054066034A840A941C3E913F9E813F8C31A
:100BAD00E913F9E813F8306904E92440F9C2AF53A9
:100BBD00E67F759100C3E498F594E499F5957591E8
:100BCD0004D26043E680D2AF22D264754300752013
:100BDD0000306C03752040020BF5D264754300752F
:100BED002040306C0375200078017901206620E5E6
:100BFD002D54066002C2647914E541C313700104DB
:100C0D00F8C3941440027814306904781B791B20C2
:100C1D006010E543600C306903D53404D26D819FBB
:100C2D0071960543E59B5440B520028189306909D1
:100C3D0008C3E899400118811C20640A08C3E8998B
:100C4D00400261F5811CC264C2AF53E67F7591000D
:100C5D003066127594007595F8759104D26043E66F
:0F0C6D0080D2AF61F5E5417EFFC3334005C3334D
:100C7C004001FEC3E49E759400F5958166C3E5338F
:100C8C009401500261F530640261F5D802819D81B6
:100C9C001CC26DC2AF53E67F759100855394855489
:100CAC0095759104854D92854E93D26043E680D222
:100CBC00AFE52D54066008206A020533020CDB30C8
:100CCC006D0D206C0A206407158115810215D62242
:100CDC0078003064027801E53775F007A4F9E5F087
:100CEC0028F5F0E9A2F013A2F113A2F213F537C321
:100CFC0094785003753778C3E53795384007D2653B
:100D0C00E57BF45290306002A111854F928550938F
:100D1C00D26043E68022207D1AC2AF754202C29196
:100D2C00C295D292306204D293D290D2AF759F11F9
:100D3C00020F5FC2AF754202C291C293D290306271
:100D4C0004D295D292D2AF759F11020F5F30724BC5
:100D5C00207D24C2AF75420390013D757B02C29089
:100D6C00C290306206D294D291A17BC294D291D21D
:100D7C00AF759F01020F5FC2AF75420390013D75C5
:100D8C007B02C292C292306206D294D291A19FC2CF
:100D9C0094D291D2AF759F21020F5F207D1CC2AF00
:100DAC00754203900119757B02C290306204D29493
:100DBC00D291D2AF759F01020F5FC2AF7542039003
:100DCC000119757B02C292306204D294D291D2AFD7
:100DDC00759F21020F5F207D1AC2AF754204C2922B
:100DEC00C293D290306204D294D291D2AF759F212B
:100DFC00020F5FC2AF754204C290C295D2923062AC
:100E0C0004D294D291D2AF759F01020F5F30724B16
:100E1C00207D24C2AF754205900131757B04C291CF
:100E2C00C291306206D295D292C13BC295D292D277
:100E3C00AF759F11020F5FC2AF75420590014975E6
:100E4C007B01C291C291306206D293D290C15FC233
:100E5C0093D290D2AF759F11020F5F207D1CC2AF51
:100E6C0075420590010D757B04C291306204D295D8
:100E7C00D292D2AF759F11020F5FC2AF754205902F
:100E8C000125757B01C2913062E8D293D290D2AF2A
:100E9C00759F11020F5F207D1AC2AF754206C2907A
:100EAC00C294D291306204D295D292D2AF759F0186
:100EBC00020F5FC2AF754206C292C294D2913062E9
:100ECC0004D293D290D2AF759F21020F5F30724B38
:100EDC00207D24C2AF754201900149757B01C292FD
:100EEC00C292306206D293D290C1FBC293D290D2FE
:100EFC00AF759F21020F5FC2AF7542019001317532
:100F0C007B04C290C290306206D295D292E11FC28D
:100F1C0095D292D2AF759F01020F5F207D1CC2AF9C
:100F2C00754201900125757B01C292306204D29307
:100F3C00D290D2AF759F21020F5FC2AF7542019064
:100F4C00010D757B04C290306204D295D292D2AF5F
:100F5C00759F01C2652290010B757B00C292C291F4
:100F6C00C290C292C291C290C26222788076090865
:100F7C0076090876040876FF0876030876FF08766B
:100F8C000A087603087601087601788C76010876D3
:100F9C00FF0876FF0876FF0876FF0876FF087603D1
:100FAC000876FF0876FF0876FF0876250876D008C5
:100FBC0076280876500876040876FF0876020876BC
:100FCC000008767A0876FF08760108760108760024
:100FDC00087603087600227887E6FFC272BF030208
:100FEC00D2727888E6C394036008C27DE630E102D1
:100FFC00D27DC27E7889E630E102D27EC3EF9402C4
:10100C006008758E01D27302101B758E00C273229C
:10101C007880E6149000809378A5F67881E6149099
:10102C0000809378A6F67886E61490008D9378A7C6
:10103C00F67886E6F539C394025003753902789C2C
:10104C00E67538FFB402037538A0B4030375388213
:10105C0078A3E61490009A93F566120F6222227818
:0F106C0096E6FA7897E6FB7888E6B40305C3EBBF
:10107B00940EFB307F047A007BFFC3EB9AFCC39486
:10108B008250027C827572000572EC8572F0A4C3EB
:10109B00E5F0947D40F222D27F116B12059E120572
:1010AB009E7A007B007C10120594E55C2AFA740092
:1010BB003BFBDCF37C04C3EB13FBEA13FADCF7FE1C
:1010CB00C27F116B22757C00757D00E5EF20E60376
:1010DB007520000520903FFFE520146006901FFF50
:1010EB001460009304600375EF1653D9BF7581C06C
:1010FB0043FF8012058F75EF0643B203E5B324025D
:10110B0020E70DF521E5E320E0068521B343E3015C
:10111B00120F627580FF75A40075F19175D47F7500
:10112B00900075A53F75F23F75D50075A60175E268
:10113B0041120F62E4F8F6D8FD756801120F7712B1
:10114B00162D78988673753001C2AF1205A812055B
:10115B00B812059E1205BF12059E1205C612059EFA
:10116B00C2AF757C00757D0078FA79FA308707D9A4
:10117B00FBD8F7021C00120FE3111C116A116B78DC
:10118B00988673120F6275881075890275C824755D
:10119B00910475D84075A82275B80275E690759BB9
:1011AB0080759D0075D10E75BC5875BB0E75BA1147
:1011BB0075E88012058FD2AF1208A475360053DA8A
:1011CB00CF207E0343DA20307E0343DA1043DA016B
:1011DB00C2D8C2711205A8D2617B037A0CE55B7091
:1011EB00077A0CDB0302116B12059E2070030211B0
:1011FB006BC270E55CC3940240E1E52F541F855E22
:10120B005DF55EB55DD5DAD5C26153DACF207E03CD
:10121B0043DA20307E0343DA10C2D8C27178A2E6DB
:10122B007008D274E52F54E0F52FC27575290012A2
:10123B0005A3307409C3E529940A4002D27512053F
:10124B009478023074027800C3E55C9840F0C2AF2A
:10125B001205B81205B81205B8D2AF1205A8754C15
:10126B00007888E6B40302615F120594788CE6C3BC
:10127B009401500302135FE530C394015003021332
:10128B005F757CA5757DF1207435C3E55C94FF50CB
:10129B000302135FC2AF1205CDD2AF1205A3C3E594
:1012AB005C940150EFC2AF1205B81205991205B844
:1012BB00D2AF1205A3C3E55C94FF40E90217D97FB7
:1012CB0002D27F116B1205A3C2AFC27F116BAE5C52
:1012DB00C3E55C947FD2AF5002616F12058FC2AF32
:1012EB001205CDD2AFDFDA11A2C3EE7897F6120555
:1012FB00A812175C7F0AD27F116B1205A3C2AFC273
:10130B007F116BAE5CC3E55C947FD2AF50E61205E8
:10131B008FC2AF1205B81205991205B8D2AFDFD63E
:10132B0011A2EE24037896F6F87997E7C3948240DE
:10133B0003985006E824827897F61205A812166FC8
:10134B0012178B1205A3116BC3E55C94FF5002417E
:10135B008C0217D9757C00757D00C3E55C954C40FC
:10136B0003855C4C1205A378017988E7B4030278F6
:10137B0005C3E55C984002416CC2AF1205CD120566
:10138B00CD1205CDD2AF1205A8753000E4F531F5BD
:10139B00320531E531F4703F0532789AE67819144D
:1013AB006012783214600D787D14600878FA14603E
:1013BB0003753200C3E53298401D120F6212058F80
:1013CB00153275310078998673C2AF1205CDD2AF45
:1013DB00789886731205A3120599E52A7005307467
:1013EB0002216B78012074027806C3E55C9840A15A
:1013FB007888E6C3940360031205A3E52A70030201
:10140B00116BC2AF120F62E4F522F523F524F5251B
:10141B00F526F567D2AF7885E6C333F565E4F54479
:10142B00F545F546F547F548F570F52CF52DF537EF
:10143B0075700875BB1012058F1208A830EDFDA84A
:10144B00BDA9BEE97001F888711208AC75700875FA
:10145B00BB10120FE3C2AF7561FF12094285226107
:0E146B00852262852263D2AF752201752401AD
:10147900752501752601856069756A017888E6B464
:101489000307C27D307602D27DD268D269753300F6
:10149900120EA2120ED912096212096912096212F8
:1014A9000969120962120BE71206B6120CDC120D59
:1014B90022120969120BD6306E0312071220660335
:1014C90012085E30660312088E120CDC120D5912D6
:1014D9000969120BE7306E03120747120CDC120D73
:1014E900E2120969120BD6306E031207A5120CDC41
:1014F900120E19120969120BE7306E031208021253
:101509000CDC120EA21209691208A8120BD6120CD1
:10151900DC120ED91208AC1209693069328564618E
:10152900856462856069756A0179187A0CC3E53347
:1015390099400FC269D26A8A3585646185646302FC
:101549001558C3E55C940140030214AE0215DE3060
:101559006A1D206C1AE535147006C26AD26B81AE19
:10156900F535C3E55C940140030214AE0215DE753E
:10157900360078FA79A4E760027803C3E55F9850EA
:1015890054307404E52A604D7888E6B40317207D49
:1015990005207607A1AE307602A1AE206C07D26C89
:1015A90085646181ED78F0306C058564617820C3CC
:1015B900E54198500281AE306C1BC26CC27D307619
:1015C90002D27DD26A75351285646181AE0536E530
:1015D9005C6002A1E1753600C2AF120F627887E63E
:1015E900FE7602120FE37887EEF6E4F522F523F58D
:1015F90024F525F526F565752C00752D00D2AF1259
:1016090005A3120F6278A4E6600CC295D292C29427
:10161900D291C293D290307409C3E5369404400242
:10162900216B6197901A0D78201216B1E520B455F7
:101639000CA31216B1E520B4AA0302164F120F77B4
:1016490012166F02166E901A0378807B0A1216B171
:10165900A308DBF9901A0F788C7B191216B1A3082D
:10166900DBF9901A2822C2AF1216F41216D1901A79
:1016790000740E1216B6A374071216B6A3741512C7
:1016890016B6901A0378807B0A1216B5A308DBF9FF
:10169900901A0F788C7B191216B5A308DBF912176B
:1016A900071216E5901A2822E493F622E6438F01E1
:1016B900538FFDFFC3E583941C400122EF857CB75E
:1016C900857DB7F0538FFE22438F02438F01857CBE
:1016D900B7857DB7901A0DF0538FFC22901A0D74BF
:1016E90055D1B6901A0E74AAD1B6227A3079D0782B
:1016F90020901A40D1B1E520F709A3DAF7227A3010
:1017090079D0901A40E7D1B609A3DAF922AB74A8C7
:1017190075BB01027980BB02027981BB0302798220
:10172900BB04027984BB05027986BB06027992BBA8
:1017390007027987BB080279A3BB0902799CBB0A16
:10174900027988BB0B027989E8F7227C051205A882
:10175900DCFB22C2AF1205B81205BF1205C612057D
:10176900CD1205991205B81205BF1205C61205CD8D
:101779001205991205B81205BF1205C61205CDD278
:10178900AF22C2AF1205CD1205C61205BF1205B8A8
:101799001205991205CD1205C61205BF1205B81218
:1017A90005991205CD1205C61205BF1205B8D2AFAB
:1017B90022AE74AF75C2AF1205B81205B81205B8DA
:1017C900120599DEF21205CD120599DFF8D2AF2282
:1017D900F15CF154F154757401757501757600F178
:1017E900BA7C05AD5C1205A8C3ED955C70F5C3E53F
:1017F9005C9401400AC3E55C94FF40370218191252
:10180900171612166F12175CC2AF75EF161217541E
:10181900DCD10576C3E5769403500280C2121754D1
:101829000575E5741490009F93F808C3E575985001
:101839000280A91217541217540574C3E574940C45
:1018490050028095120F7712166FC2AF75EF1612FC
:02185900175422
:0319FD000210D005
:101A00000E0715090904FF03FF0A03010155AA0186
:101A1000FFFFFFFFFF03FFFFFF25D0285004FF0259
:091A2000007AFF0101000300FF40
:101A400023454D41585F4C746E675F32304123200F
:101A500023424C48454C492346333930232020202B
:101A60002020202020202020202020202020202076
:101C0000C2AFC2D353D9BF7581C043B20343FF8073
:101C1000752438752503B1DC7529A5752AF175E29F
:101C20004043F18053A47F75D4FFD2877DFA7803B7
:101C300079E67C10752200752300901DE97B0675FE
:101C400024987525013087028145208708D8FBD963
:101C5000F9DCF781B7308708D8FBD9F9DCF781B711
:101C6000B19CE493A3C39A6004DDC381B7DBDBB10D
:101C70008E6002812E7B08E493FAA3B16FDBF87AC1
:101C800030B16F752200752300B18EEAFCEBFDC305
:101C9000ED94FE400EB18E8A278B28ED30E0048A49
:101CA000828B83B18E7AC270D8C3ED94FE601950D6
:101CB000CEBD002BEC600F7520007521FF7529004B
:101CC000752A000200008100A827A9280809D80465
:101CD000D90281DCB192EA89AAF281CE0D81A3C337
:101CE000ED94035053EDA2E092007AC5C3E58294CF
:101CF00000E583941C508A200010438F02438F011B
:101D00008529B7852AB7F0300029A827A92808090E
:101D1000438F01538FFDD804D902A133C3E58394C7
:101D20001C4003A3A11689AAE28529B7852AB7F02A
:101D3000A3A116538FFC817F7AC1BD030CE493A34A
:101D4000FAB153DCF8B14B817F8181AA22AB23B178
:101D50006FEBFAEA6222752608C3E52313F523E543
:101D60002213F52250066323A0632201D526EAB18F
:101D7000DCB1DC75260AEAF4200102D287300102C8
:101D8000C287B1DCC3134002C201D526EB22B19257
:101D9000EAFB208702A192308702A197752608AE40
:101DA00024AF25C3EF13FFEE13FEB1E0B1DCC3EAAD
:101DB000133087024480FA30E703632201C3E5232E
:101DC00013F523E52213F52250066323A0632201B5
:101DD000D526D9E52265236523F52222AE24AF2539
:101DE0000E0FDEFEDFFCD20122424C48656C6934E6
:071DF000373163F390060197
:00000001FF
